:10000000AC018E28AC16AC1EAC122C190C28FE3993
:10001000AD002C15031089282C1A142892002C16D8
:100020002B20031819281208322003181928AC1E97
:100030008928242049202C112C12AC11300884006E
:100040002E08841780042A28300884002E09800591
:100050008417800508001E204920242045202D08F3
:10006000AC1901388E0008308F008E0D03181E2049
:10007000031C2420492045208F0B35281E204920B1
:10008000300884002E080005FF3E310884002F0947
:100090002728310884002F08800484172F09800541
:1000A0002A288F018E00FF308E07031C8F07031C48
:1000B000892803308D00DF305F2053288D01E83E12
:1000C0008C008D09FC30031C68288C0703186528F8
:1000D0008C0764008D0F65280C186E288C1C722804
:1000E000000072280800103094008D018C01930CE0
:1000F000920C031C81280E088C070F0803180F0FA1
:100100008D078D0C8C0C910C900C940B772810089B
:1001100089288313031383126400080083160614CE
:1001200086150615861406168616061786170510F8
:1001300085108312C230B600E030B4004730B500FD
:100140008030861F03019E000030861F03019F0040
:100150001E08FF3C9E001F08031C013E003C9F0040
:100160004030061F0301A0000030061F0301A1005C
:1001700020081E02A0002108031C013E1F02A1004E
:100180002030861E0301A2000030861E0301A3005A
:1001900022082002A2002308031C013E2102A30022
:1001A0001030061E0301A4000030061E0301A50046
:1001B00024082202A4002508031C013E2302A500F6
:1001C0000830861C0301A6000030861C0301A7002E
:1001D00026082402A6002708031C013E2502A700CA
:1001E0000430061D0301A8000030061D0301A9000C
:1001F00028082602A8002908031C013E2702A9009E
:100200000230861D0301AA000030861D0301AB00E9
:100210002A082802AA002B08031C013E2902AB0071
:100220002A080618FF3EB7003708920093010830ED
:100230008E008F0173209E0011089F0034081E0756
:10024000B20035080318013E1F07B3000530B000A7
:100250000230AE000530B1000130AF003608042096
:1002600033080420320804208E30022001308F0031
:0A027000F4305220A02863003B295F
:02400E00F73F7A
:00000001FF
